:03000000020030CB
:03000B00020141AE
:10003000310820B002515A300021C200EA90031B5F
:1000400093FBBB0A05115E02005BBB0B05118F021F
:10005000005B00A60308B878027870020037787059
:10006000760008B878FA787022E5301475F008A4A4
:10007000F53086F0E53051A35136080530B878F2F6
:10008000115EC201C20220B103D29622C29622782A
:10009000702001D57530017B00EB517386F0B5F00F
:1000A000300B08B878F3115EE530B40107D203D203
:1000B0000231712274405173B40005B2B1B296227C
:1000C000C28CD2B1C2965119115ED296C2B1D28CF5
:1000D000220B08B878FB78700530BB40BC115EA2DB
:1000E000969204752180C296300905300A02D29694
:1000F0005136514651365146513651465136513698
:10010000D521E3A204929622D2B0D2B7D290D29156
:10011000D292C295C294C293D296C2007A00C2B162
:10012000C202C203C201753401115E758901C28821
:10013000C2A8D28CD2A97532257533FF514CD2AFEB
:1001400022758A71758CB2C0E0C0F031C8D5341107
:1001500020030675340602015C753401300202B2D8
:1001600096200208D53605115E753699D0F0D0E09C
:10017000323000FDC200EA90031B93FBBB0B03026D
:1001800001B6BB00030201B6BB0A030201B6BB09FC
:1001900030C2033000FBC200EA90031B93FBB40A99
:1001A000030201B6B40B030201B675F002A4C5F058
:1001B000744051A35136C20220B103D29622C29696
:1001C00022D201C2038B3022D294D293C29551061F
:1001D00075F000701CD295C294510675F004701130
:1001E000D294C293510675F008D2937004E40201D0
:1001F000F325F0B5020122CA700BD200753699C200
:100200008C5146D28C22740130B70D043090090411
:1002100030910504309201E4227531FF7535FF7489
:10022000405173D531FD7531FFD535F77531FF7507
:1002300035FFD5E0EE227531FF753515D531FD75E9
:1002400031FFD535F722753225753315B2B3D53266
:10025000FD753225D533F5D2B322753700E53790D9
:100260000328513693F5F0E53751A30537E537B448
:1002700041F022C0F0F5F051FE402574A04400C2C8
:10028000E051C74019E5F051C7401351FE401174C9
:10029000A04400D2E051C7400551E9C38002711269
:1002A000D0F02251FE401FC0E074A04400C2E051D3
:1002B000C7400FD0E0C0E051C74007E5F051C7404C
:1002C00001C37112D0E022C0F075F0083392B5007E
:1002D000D2B400C2B4D5F0F4D2B50000D2B400005C
:1002E0000000A2B5C2B4D0F022D2B5C0F075F008BB
:1002F000D2B400A2B533C2B4D5F0F5D0F022D2B555
:10030000D2B430B50B30B408C2B500C2B4C380015A
:10031000D322C2B500D2B400D2B522FF0104070A2D
:10032000020508000306090B010203040000000097
:1003300002020202000000000303030300000000A9
:100340000404040400000000050505050000000089
:100350000606060600000000070707070000000069
:0903600008080808000000000272
:00000001FF
